:10000000B20154290408A700061086108610831632
:10001000061086108610870183122708B2182B2835
:100020003A30A100983017213330A6003E2013301B
:10003000A100883017213E20643016213E20643014
:10004000162138302A200C302A2006302A20B214FB
:1000500027082B283214A600321C39288610033CAE
:10006000031C3E283E200730A100D0301721031486
:1000700008003214FE3C03194F2986140614260882
:1000800087000000321006103230162103140800D9
:10009000003803194F29A80020088400211883176D
:1000A000A001A101A81B5C280008A000A81C4F29E2
:1000B000840A0008A1004F29F4200005031DA00AAE
:1000C0004F296400772003186128B620A801083062
:1000D000A300B72077200318A80AAB1EA801A20C22
:1000E000A30B6928AB1AA213B72022080800360810
:1000F0008400340884178004841300052B1B340605
:10010000FF3E0800A401A501B3124A21D33E031902
:10011000B3162D3EC63E031885280A3E031C8528CB
:10012000A2000310240DA000250DA100200DA10D9B
:10013000A4070318A10A2108A507A40DA50D2208EC
:10014000A4070318A50AA9030319AD284A21C63E2E
:100150000318AD280A3E03189028B31EB428A4093A
:10016000A509A40A0319A50A24084F2933172B0847
:100170001F39003EA1002A080E3E0318A10A331FB2
:1001800017293313A000023029211729B313290896
:100190000319B3170530A8002730A3001030DC2066
:1001A0000330A300E830DC20A3016430DC20A3018D
:1001B0000A30DC202408E328A2002508A100240836
:1001C000A0002E212008A000A8030319B3132908BA
:1001D0000319ED282802031808002008031DB31393
:1001E000B31B0800303E4A2901308A00280807392D
:0201F0000029E4
:10020000820701340234043408341034203440347A
:100210008034A301A200FF30A207031CA307031C24
:100220004F290330A100E63017210B29A101FC3E24
:10023000A000A109031C2229FF300000A007031819
:100240001D29A0076400A10F1C2908000310A10CA0
:10025000A00CFF3E0318262920084F29A501A40160
:100260001030A600210DA40DA50D2208A40223081C
:10027000031C230FA502031844292208A4072308FE
:100280000318230FA5070310A00DA10DA60B3229FB
:1002900020084F29840031088A0030088200831327
:1002A0000313831264000800831607309F00831233
:1002B000C401051483160510831285148316851056
:1002C0008312851583168511831206118316061174
:1002D000051485148515061583128512831685125B
:1002E00083120130A300F4300A21640005187A2932
:1002F00044107B294414640085188029C410812986
:10030000C4146400851986294411872944156400A2
:1003100004304402031C91290430C4024E30C6004C
:1003200093295430C6004408A200033C031CB8299A
:100330000310220DA207A821A000A20AA821A10053
:10034000A20AA82148202008C0002108C100B8291D
:1003500001308A00220882072034003400342D3412
:10036000033400348C340134003454340034003409
:100370004408A200033C031CDD290310220DA20740
:10038000CD21A000A20ACD21A100A20ACD214820A2
:100390002008C2002108C300DD2901308A0022089C
:1003A000820700344B340034B034043400346034F9
:1003B00009340034803425340034640046084E3C4F
:1003C000031DE32941177C232030CA000630B60004
:1003D0000430B4004008AA004108AB0061200D3C85
:1003E000031DEE296120CC000630B6000430B400B5
:1003F0004008AA004108AB006120CA0064004A0816
:100400005C3C031D042A3A2A64004A085D3C031D33
:100410000A2A822A64004A085B3C031D102A942A97
:1004200064004A08083C031D202AFE3003201030D7
:10043000032020300320FE30032010300320392A0F
:1004400064004A08093C031D312A0130C9006400D8
:10045000063049020318302A20300320C90F272A0A
:10046000392A64004A080D3C031D372A392A4A08F4
:100470000320F4290630B6000430B4004008AA0076
:100480004108AB000330A9006130B000B101822007
:10049000CB0064004B08013C031D552AFE300320AD
:1004A000013003201E300921812A64004B08803C62
:1004B000031D5F2AFE30032080300320812A640060
:1004C0004B08C03C031D692AFE300320C0300320C6
:1004D000812A64004B08943C031D732AFE300320DC
:1004E00094300320812A64004B08D43C031D7D2AEC
:1004F000FE300320D4300320812AFE3003204B0835
:100500000320F4290630B6000430B4004008AA00E5
:100510004108AB000330A9006130B000B101822076
:10052000CB004B080320F4290630B6000430B40099
:100530004008AA004108AB000230A9006130B000B9
:10054000B1018220CB0064004B081E3C031DAD2A84
:100550008611831686118312722B64004B081F3C90
:10056000031DB72A8615831686118312722B640029
:100570004B08283C031DC12A06128316061283125B
:10058000722B64004B08293C031DCB2A06168316E8
:1005900006128312722B64004B08323C031DD52ACD
:1005A0008612831686128312722B64004B08333C2A
:1005B000031DDF2A8616831686128312722B6400AF
:1005C0004B083C3C031DE92A0613831606138312CD
:1005D000722B64004B083D3C031DF32A061783165B
:1005E00006138312722B64004B08463C031DFD2A40
:1005F0008613831686138312722B64004B08473CC4
:10060000031D072B8617831686138312722B640033
:100610004B08623C031D6C2B0630B6000430B4005E
:100620004008AA004108AB000330A9006130B000C7
:10063000B1018220C5000230A9006130B000B101D3
:100640008220B8000230A9006130B000B1018220E0
:10065000B9000230A9006130B000B1018220BA00B7
:100660000230A9006130B000B1018220BB0002302D
:10067000A9006130B000B1018220BC000230A900A5
:100680006130B000B1018220BD000230A9006130AC
:10069000B000B1018220BE000230A9006130B0007C
:1006A000B1018220BF00FE30032045080320380836
:1006B0000320390803203A0803203B0803203C08A4
:1006C00003203D0803203E0803203F080320FE309E
:1006D000032080300320722B64004B08633C031D11
:1006E000722B4524F4296300732BFE300320013064
:1006F00003201E3009210800851683168512870104
:1007000083120130A3002C300A21FE300320403038
:1007100003200030032004300320023003201F3068
:100720000320023003200430032000300320003077
:100730000320FE30032080300320FE3003204830A9
:1007400003200030032004300320083003201F3032
:100750000320083003200430032000300320003041
:100760000320FE30032080300320FE300320503071
:10077000032000300320043003200E300320153006
:100780000320043003200430032000300320003015
:100790000320FE30032080300320FE300320583039
:1007A00003200030032000300320043003200430F5
:1007B0000320153003200E300320043003200030C6
:1007C0000320FE30032080300320FE300320603001
:1007D00003201F300320113003201130032011307B
:1007E00003201130032011300320113003201F306B
:1007F0000320FE30032080300320FE3003206830C9
:100800000320043003200E3003201F30032000306B
:100810000320003003201F3003200E30032004305B
:100820000320FE30032080300320FE300320703090
:10083000032002300320063003200E3003201E3038
:1008400003200E3003200630032002300320003046
:100850000320FE30032080300320FE300320783058
:100860000320083003200C3003200E3003200F300B
:1008700003200E3003200C3003200830032000300A
:100880000320FE30032080300320FE30032001309F
:1008900003201E300921FE30032080300320533016
:1008A000032065300320723003206930032061305B
:1008B00003206C30032020300320433003204C30D1
:1008C00003204330032044300320203003207630BF
:1008D0000320313003202E30032030300320FE303F
:1008E0000320C030032042300320613003207530E4
:1008F0000320643003203A300320203003204608D0
:100900000320A9014208A4004308A5000230B0005A
:0E091000B101C620FE30032002300320080093
:02400E00753FFC
:00000001FF
